:020000040000FA
:020000007A2D57
:08000800F1000308F2000A08F0
:10001000F300831203130000CB0F1428CC0F142815
:100020005F14CD0F14285E14213081002A08003E91
:1000300003192F28241C2D28051656200130602076
:1000400000001E30A10005120730602005160630A2
:100050006020A10B232800003C2856203C28492082
:10006000452064206A2078204D200E30A1000F30FA
:100070006020A10B372800000B11051273088A00BD
:1000800072088300F10E710E09003410851E3414BD
:1000900008002D1085192D1408004A082B02031C96
:1000A00054282B08CA000800000008002410AA03E6
:1000B0000310A80CA70CA60CA50C03182414080008
:1000C000D300D30B6128080003102B0DAC00712066
:1000D000B200080003102B0D013EAC007120B300EC
:1000E000080000308A002C087C3E03188A0A82002F
:1000F00032088A00330882000034C4340034CC341F
:100100000034D4340034DC340034E4340034EC34CF
:100110000034F4340034FC340134043401340C343D
:100120000134143401341C340134203401342C34AF
:100130000134303401343C340134403401344C3423
:100140000134503401345C340134603401346C3493
:100150000134703401347C340134803401348C3403
:100160000134903401349C340134A0340134AC3473
:100170000134B0340134BC340134C0340134CC34E3
:100180000134D0340134DC342D18C9280730AB00D9
:10019000DE290130AB00DE292D18D1280030AB005C
:1001A000DE290230AB00DE292D18D9280030AB0043
:1001B000DE290330AB00DE292D18E1280430AB0026
:1001C000DE290330AB00DE292D18E9280030AB0012
:1001D000DE290530AB00DE292D18F1280B30AB00ED
:1001E000DE290030AB00DE292D18F9280030AB00E5
:1001F000DE290030AB00DE292D1801290830AB00C4
:10020000DE290030AB00DE292D1809290930AB00AA
:10021000DE290030AB00DE292D1811290A30AB0091
:10022000DE290030AB00DE292D1819290A30AB0079
:10023000DE290030AB00DE292D08B100AB0ADE2933
:1002400031082D06031D2629AB01DE292D1830109B
:100250002D1C3014AB0ADE292D08B100AB0ADE29B3
:1002600031082D06031D3629AB01DE292D182F126A
:100270002D1C2F16AB0ADE292D08B100AB0ADE2992
:1002800031082D06031D4629AB01DE292D18AF11BB
:100290002D1CAF15AB0ADE292D08B100AB0ADE29F3
:1002A00031082D06031D5629AB01DE292D182F110B
:1002B0002D1C2F15AB0ADE292D08B100AB0ADE2953
:1002C00031082D06031D6629AB01DE292D18AF105C
:1002D0002D1CAF14AB0ADE292D08B100AB0ADE29B4
:1002E00031082D06031D7629AB01DE292D182F10AC
:1002F0002D1C2F14AB0ADE292D08B100AB0ADE2914
:1003000031082D06031D8629AB01DE292D18AE12FA
:100310002D1CAE16AB0ADE292D08B100AB0ADE2972
:1003200031082D06031D9629AB01DE292D182E124A
:100330002D1C2E16AB0ADE292D08B100AB0ADE29D2
:1003400031082D06031DA629AB01DE292D18AE119B
:100350002D1CAE15AB0ADE292D08B100AB0ADE2933
:1003600031082D06031DB629AB01DE292D182E11EB
:100370002D1C2E15AB0ADE292D08B100AB0ADE2993
:1003800031082D06031DC629AB01DE292D18AE103C
:100390002D1CAE14AB0ADE292D08B100AB0ADE29F4
:1003A00031082D06031DD629AB01DE292D182E108C
:1003B0002D1C2E14AB0ADE29AB0154140800C20117
:1003C000C3010830C4000310C60CC30DC20DC50C18
:1003D000C30DC20DC40BE3290800A601A701A801A3
:1003E000A030A500D909591C26145918A614571E67
:1003F0002615571AA615D71D2616D719A616571D46
:1004000026175719A617D71C2714D718A714571C37
:1004100027155718A715D81E2716D81AA716581E1D
:100420002717581AA717D81D2814D819A814581D0B
:1004300028155819A815D81C2816D818A816581CFD
:1004400028175818A8172130AA000800C700000074
:10045000C70B272A0800CB01CC01FD30CD000530A9
:10046000E5000800CE0A4E08103C0319CE014E08E4
:10047000DA002B220800CE034E08013E031D432A5A
:100480000F30CE00DA002B2208002E08CE00DA0052
:10049000F03E031C4F2A0F30CE024E08482A2B2272
:1004A00008008B1383160313073085043F3087043D
:1004B00083120313F8308505C030870583160313B4
:1004C00074088505750887058312031335088504AC
:1004D000360887048B1708000730F4043F30F50412
:1004E000F830B505C030B60508004808C1006C22D8
:1004F000BA19F410BC197411BE197510C019F51091
:10050000B7197511B71AF511371B7512371AF5128D
:10051000741035145122B03026226C22B91974108F
:1005200039187411B91875103919F5107515B91AEB
:10053000F511391B7512391AF512F410B514512240
:10054000B03026226C22BB1974103A18F410BB1874
:1005500075103B19F51037187511BB1AF5113B1BB7
:1005600075123B1AF512741135155122B03026223E
:100570006C22BD197410BA18F410BC1874113D190E
:10058000F510B7187511BD1AF5113D1B75123D1AFE
:10059000F512751036145122B03026226C22BF1984
:1005A00074103A19F4103C1974113E19751037196A
:1005B0007511BF1AF5113F1B75123F1AF512F51090
:1005C000B6145122B03026226C22B8197410F414DB
:1005D00038187411B81875103819F5103E18F5113F
:1005E0003C1875124018F512751136155122B030AD
:1005F00026226C22B81A7410BA1AF410BC1A74119C
:10060000BE1A7510C01AF5103D187511BD18751277
:100610004019F512F511B6155122B03026226C2280
:10062000381B74103A1BF4103C1B74113E1B7510E0
:10063000401BF5103B187511BE18F511C018F512C6
:10064000751236165122B03026226C22381A7410D8
:100650003A1AF4103C1A74113E1A7510401AF5102B
:100660003F1875113F19F511BF187512F512B6161E
:100670005122B0302622C10B772A08004E08013ED5
:10068000B700B801B901BA01BB01BC01BD01BE018F
:10069000BF01C001FF305B18BF007F30C80075226A
:1006A00008004E08031D5F2B03019E23D100DB01D0
:1006B000D11B5B145108031D742B3222512B0530C2
:1006C000CF00C430D00003104E0DF6008B13BD25B3
:1006D0008B17D10003104E0D013EF6008B13BD2584
:1006E0008B17D0005108CF0008004E08031D7B2B4C
:1006F000760A9E23852B0A08DC0076088B13BD251D
:10070000DD005C088A008B175D08F60A0800831676
:1007100003131C158B1376089B0077089A0055303D
:100720009D00AA309D009C148B1783120313FF3089
:10073000B700B8003F30C8007522080083160313C5
:100740009B009C131C141A08831203130800F60163
:10075000D501D601E8010530F600FF30B700B8003A
:10076000B900BA00BB00BC00BD00BE00BF00C000A5
:100770007F30C800752276089E23F70077080C2585
:100780001F30C8007522D40177080C250230C8003C
:100790007522541CC42BAF08031DC42B10302E022D
:1007A000031DE02B55188723D501F60A7608013E74
:1007B000031DDC2BFE30F60076089E23F700BE2BCF
:1007C00011302E02031DF22B55188723D501F60395
:1007D0007608053C031CEE2B0530F60076089E23B8
:1007E000F700BE2B20302E02031D002C0130F70233
:1007F00077081F3C031CFE2B7A30F7005514BE2BE4
:1008000021302E02031D0E2C0130F70777087A3CA9
:1008100003180C2C2030F7005514BE2B01302E028B
:10082000031D162C0130F7005514BE2B02302E028A
:10083000031D1E2C0230F7005514BE2B03302E0270
:10084000031D262C0530F7005514BE2B09302E024F
:10085000031D2E2C0030F7005514BE2B00302E0245
:10086000031D3F2C7708603C03183A2C2030F70218
:1008700068143D2C2030F707E8015514BE2BC42B1B
:1008800003019E23D100D11F482CD113DB014A2C38
:10089000D1175B14F6015108F70087233E233E234E
:1008A00008005123F6017523D2007523C900C90A37
:1008B000541C762C07302F02031D612C4522D401D5
:1008C000512CAF08031D762C20302E020319322242
:1008D00021302E0203193B2200302E020319CE01D3
:1008E0000C302E0203194024D401512C341C812CCD
:1008F0003E233E23341C812C32223E2334187C2C90
:10090000512C013052020319AB2402305202031958
:10091000C024033052020319C624043052020319C2
:1009200052254908C80075225F189F2C2A08003EEE
:10093000031D9F2C0730D7005A08D800ED215E1CFC
:10094000A82CDE015B1CA82CFD30CD003222512CDE
:10095000C01F582C512C7523B7007523B800752380
:10096000B9007523BA007523BB007523BC0075233D
:10097000BD007523BE007523BF007523C0000800AD
:1009800063257523BF007523C00008007523E000B0
:10099000E00803190A2D203060020318D22C6008E9
:1009A000E500C62C2030E0024430E2000A30E300CB
:1009B0006008E2070318E30A0310E00DE00D0318D6
:1009C000E30A6008E2070318E30A8B137425E100C9
:1009D0005C088A008B1763256108BF006108C000AE
:1009E000651CBF01651DC001E518BF09E519C009F7
:1009F0000130E2070318E30A4908C8007522C01352
:100A0000E11FE52C6325BF01C001E518BF09E51909
:100A1000C0090B2DC0170800E700E708031D132DC0
:100A20007C30E700222D2030670203181C2D670858
:100A3000E5007B30E700222D7B306702031C222D6E
:100A40007D30E7002030E7024430E2000A30E30066
:100A50006708E2070318E30A0310E70DE70D031820
:100A6000E30A6708E2070318E30A0530E6008B1380
:100A70007425E1005C088A008B1763256108BF00BC
:100A80006108C000651CBF01651DC001E518BF09F4
:100A9000E519C0090130E2070318E30AC013E60BA9
:100AA000372D08007523E000E0080319612D203080
:100AB000600203185E2D6008E500522D60080C25C9
:100AC0000B2DC01708003908B7003A08B8003B08DA
:100AD000B9003C08BA003D08BB003E08BC003F0816
:100AE000BD004008BE0008000A08DC0063088A0058
:100AF0006208820085018701F401F501B501B601A4
:100B0000AB01AD01B001AF01AE01B101CA0181017C
:100B1000B401CB01CC01FD30CD000530E500FF3044
:100B2000C600C501DF2100000730990083160313BA
:100B3000823081000F168F160F178113F41695015E
:100B400095169101073099008112831203138B16B9
:100B50008B17CE01F415CE01FF30B700B800B900F5
:100B6000BA00BB00BC00BD00BE00BF00C0007F30AB
:100B7000C8007522341C512CA72B4F088A00760818
:100B8000500703188A0A82000534E4340534E4343B
:100B90000534F43406341D34063497340634A9344D
:100BA00007349B3408340B340834353408345A3451
:100BB000083498340834B8340834CA340934263434
:100BC00009348C340934CA340434303404344434A1
:100BD000753463344B346F346E3420340134313423
:100BE0003534203420340034033420340434443485
:100BF000753463344B346F346E34203405343134FF
:100C0000353420340134203442346534773461344F
:100C10007234653420347434683465342034493493
:100C200064346534733420346F346634203444348F
:100C3000753463346B342134003401343034073478
:100C400000340034023400340034003400341C34E6
:100C500000340734003400340034003401340034EC
:100C600000340E34003407340034003400340034CF
:100C7000003400340234073400340E3400340034BD
:100C8000003400340434003400340E3400341C3496
:100C900000340034083400340034003400341C3490
:100CA00000341C3400340034003400341034003478
:100CB0000034383400341C34003400340034003440
:100CC00000340034203470340034383400340034BC
:100CD0000034003440340034003470340034703454
:100CE00000340034203400340034003400347034D4
:100CF000003438340034003400340034103400340C
:100D00000034703400341C340034003400340034B7
:100D10000034003408341C3400340E340034003401
:100D2000003400340434003400341C348034033480
:100D3000203404347734773477342E3432344434E6
:100D40004B346934743473342E3463346F346D34FB
:100D5000003401340734F8340034003400340034F3
:100D6000003400340034003400340734C03400341C
:100D700000340034003400340034003400340034D3
:100D80003E34003400340034003400340034003485
:100D9000003400340134F0340034003400340034C2
:100DA000003400340034003400340F348034003414
:100DB0000034003400340034003400340034003493
:100DC0007C34003400340034003400340034003407
:100DD000003400340334E034003400340034003490
:100DE0000034843421340834423400340034003474
:100DF000003400340034423410348434213400345C
:100E000000340034003400340034213408344234D7
:100E10001034803400340034003400340034103492
:100E20008434213408344034003400340034003435
:100E30000034083442341034843420340034003414
:100E400000340034003400340034003400341F34E3
:100E500000340034003400340034003400340034F2
:100E600000340034F83400340034003400340034EA
:100E700000340034003400340734C034003400340B
:100E800000340034003400340034003400343E3484
:100E900000340034003400340034003400340034B2
:100EA00000340134F03400340034003400340034B1
:100EB00000340034003400340F3480340034003403
:100EC00000340034003400340034003400347C3406
:100ED00000340034003400340034103484342134BD
:100EE0000834403400340034003400340034083412
:100EF000423410348434203400340034003400345C
:100F000000340434213408344234103400340034C2
:100F10000034003400340234103484342134083472
:100F200000340034003400340034013408344234D6
:100F300010348534803401341034013400340034EA
:100F400000340034003400340034003400340234FF
:100F500000340134003400340034003400340034F0
:100F600000340434003402340034013400340034DA
:100F700000340034003408340034043400340234C3
:100F800000340134003400340034103400340834A8
:100F9000003404340034023400340134003420348A
:100FA0000034103400340834003404340034023483
:100FB0000034403400342034003410340034083419
:100FC000003404340034003400344034003420341D
:100FD0000034103400340834003400340034003459
:100FE00000344034003420340034103400340034F1
:100FF00000340034003400340034403400342034F1
:101000000034003400340034003400340034003440
:10101000003440348034013410340034003400345F
:101020000034083400340034003400340034003418
:1010300000341C340034143400341C3400340034C4
:1010400000343E340034223400342234003422345C
:1010500000343E34003441340034413400344134EF
:1010600000344134003441348034033420340534B6
:1010700053346F3420346D3461346E347934203419
:1010800042346C3469346E346B346934653473348F
:101090002C34203473346F3420346C346934743419
:1010A00074346C3465342034743469346D3465348C
:1010B0002034003401341034043420340234103429
:1010C00041340834023410340434203402341034EF
:1010D00041340834203404344134083402341034A8
:1010E00041340834203404341034023420340434BD
:1010F0004134083420340434103402340834413488
:1011000010340234203404341034023408344134AE
:101110000434203408344134103402340834413467
:101120000434203402341034043420340834C134FC
:10113000013420340034003400340034633400348B
:1011400000340034003400341034003410340034DF
:1011500000340034043400340434003404340034E3
:10116000043400340034003410340034103480343B
:101170000434303404347734773477342E343234D2
:1011800044344B346934743473342E3463346F34E0
:101190006D34003401341034003400340034003431
:1011A000003440340034003400340034003400345F
:1011B00000342034003460340034203400340034EF
:1011C00000341034003420340034703400342034BF
:1011D00000341034003410340034203400347834B7
:1011E00000342034003410340034103404342034FB
:1011F000043478340434203400341034003410348F
:101200000634203406347834063420340034103464
:101210000034103407342034073478340734203451
:101220000034103400341034073420340734783458
:1012300007342034003410340034103407342034A0
:1012400007347834073420340034903401341034B7
:1012500000340034003400340034003400340034EE
:1012600000340034003400340034003408340034D6
:101270000034003400340034003400341C340034B2
:101280001C3400341C340034003400343E34003448
:101290003E3400343E3400343E3400343E340034B6
:1012A0007F3400347F3400347F3400347F340034A2
:1012B0007F3400340034003400340034003400340F
:1012C000003400340034003400340034003400347E
:1012D0000034083400340034003400340034003466
:1012E00000341C3400341C3400341C34003400340A
:1012F00000343E3400343E3400343E3400343E3456
:1013000000343E3400347F3400347F3400347F3482
:1013100000347F340034FF3401341034013400349D
:1013200002340034013401340234423404340434CD
:1013300001340834023400340434003402340234FA
:1013400004340434003408340234103404340034D7
:1013500008340034043404340034083400341034C5
:1013600004342034083400341034003400340034A1
:101370000034103401342134083440341034003443
:101380000134003400340034013421340234423456
:1013900010348034013410340534023402340534FE
:1013A0000534023400340034003400340034003496
:1013B0000534023402340534053402340034003478
:1013C000003400340034003405340234023405346F
:1013D0000534023400340034003400340A34043458
:1013E00004340A340A340434003400340034003441
:1013F00014340834083414341434083400340034F9
:101400000034003428341034103428342834103494
:10141000003400340034003450342034203450344C
:1014200050342034003400345034203420345034CC
:1014300050342034003400345034203420345034BC
:101440005034203400340034003400342834103454
:10145000103428342834103400340034003400347C
:101460001434083408341434143408340034003488
:10147000003400340A34043404340A340A340434A2
:1014800000340034003480340034803480348034BC
:101490008034DF348034803480348034033400344A
:1014A00083348034803414343E3414343E349434E1
:1014B00024342A347F342A349234233413340834C5
:1014C0006434E2343634493456342034D0341C3455
:1014D0001C349C34803480341C342234C134803435
:1014E0008034413422349C34803480342A341C3497
:1014F0007F341C34AA3408341C348834803480345B
:101500003034F03480348034803408340834883403
:10151000803480346034E03480348034803440342B
:1015200030340834063481343E345134493445343F
:10153000BE3442347F34C034803480344234613429
:1015400051344934C6342234413449344934B634F0
:101550001834143412347F349034273445344534ED
:101560004534B9343C344A3449344934B034013414
:1015700071340934053483343634493449344934B8
:10158000B6340634493449344934BE343634B6347A
:101590008034803480343634F6348034803480347F
:1015A000083414342234C1348034143414341434E0
:1015B00094348034413422341434883480340234F6
:1015C00001345134093486343E3441345D34553469
:1015D000DE347C34123411341234FC347F34493418
:1015E00049344934B6343E34413441344134A23470
:1015F0007F34413441344134BE347F34493449343A
:101600004934C1347F3409340934093481343E34D7
:10161000413449344934BA347F3408340834083406
:10162000FF3441347F34C13480348034203440343A
:101630004034BF3480347F34083414342234C1340D
:101640007F3440344034C03480347F3402340C342E
:101650000234FF347F34023404340834FF343E341F
:10166000413441344134BE347F34093409340934BF
:1016700086343E34413451342134DE347F340934ED
:1016800019342934C6342634493449344934B234FF
:10169000013401347F34013481343F3440344034E8
:1016A0004034BF341F342034403420349F343F341E
:1016B000403438344034BF34633414340834143480
:1016C000E3340734083470340834873461345134D7
:1016D00049344534C3347F344134C1348034803498
:1016E0000134063408343034C03441344134FF34DA
:1016F0008034803402340134823480348034403485
:10170000403440344034C0340034033480348034B6
:101710008034203454345434F83480347F344434A6
:101720004434B8348034383444344434C434803499
:10173000383444344434FF348034383454345434EA
:10174000D834803404347E340534813480344834D1
:1017500054345434BC3480347F3408340434F83482
:101760008034FD34803480348034803420344034FC
:10177000BD34803480347F3410342834C434803411
:10178000FF34803480348034803478340434183426
:101790000434F8347C3408340434F8348034383475
:1017A00044344434B83480347C34143414348834AD
:1017B0008034083414341434FC3480347C340834D9
:1017C000043484348034483454345434A43480345D
:1017D00004347F348434803480343C3440344034A6
:1017E000BC3480340C343034403430348C343C34A9
:1017F000403430344034BC34443428341034283439
:10180000C4344C3450345034BC34803444346434A4
:1018100054344C34C43400343E343E343E3480348A
:101820007734413463344134F7341434223414347B
:041830002234943496
:02400E00C430BC
:104200000100030014000400200059006F00750035
:1042100020006E00650065006400200074006F00DF
:1042200020006C006500610072006E0020006800D4
:104230006F007700200074006F00200063006800AA
:1042400061006E006700650020007400680069006E
:10425000730020006D00650073007300610067004B
:104260006500200077006900740068002000790074
:104270006F0075007200200054005600200072008C
:1042800065006D006F0074006500210020000500CE
:10429000540068006500200069006E00730074001F
:1042A000720075006300740069006F006E00730097
:1042B0002000610072006500200061007400200091
:1042C0007700770077002E00320044004B00690031
:1042D000740073002E0063006F006D002E0000005C
:00000001FF
